:020000021000EC
:10F8000011241FBECFEFD0E4DEBFCDBF12E0A0E0D9
:10F81000B1E001C01D92A030B107E1F70E9439FCB0
:10F820000C940FFE0C9438FC9091C80095FFFCCF0F
:10F830008093CE0008958091C80087FFFCCF2E9A58
:10F840008091CE00089581E40E9414FC86E50E9418
:10F8500014FC82E50E9414FC82E40E9414FC8FE4F4
:10F860000E9414FC8FE40E9414FC84E50C9414FCA8
:10F870000895CF93DF9300D000D000D0CDB7DEB78E
:10F880008FEF87B998B188B984B995B185B98AB92C
:10F890009BB18BB987B18B6087B988B1847F88B9F8
:10F8A000299A439AF894A89584B7877F84BF80915A
:10F8B0006000886180936000109260000C98149A38
:10F8C0001092CD008AE08093CC0088E18093C9003B
:10F8D00086E08093CA00049B04C01498E0E0F0E046
:10F8E00009952E9880E090E02091C80027FF0CC079
:10F8F0002091CE00233541F40E9423FC712C1D82FF
:10F900001C82B1E16B2E0EC0803DF7E09F0710F026
:10F9100014982998EFE4F3EC3197F1F700C0000058
:10F920000196E2CF0E941BFC813611F489E55EC18D
:10F93000813449F40E941BFC382E212C0E941BFCB0
:10F940009101282B90C0823629F489E50E9414FC8D
:10F9500081E020C1823409F089C00E941BFC582E2E
:10F96000412C0E941BFC8201082B0E941BFC982F3B
:10F97000A0E0EA2EA1E0FA2EC12CD12CC016D106AF
:10F9800028F49E830E941BFC9E8101C08FEFF7012B
:10F9900081937F01FFEFCF1ADF0AC11421E0D20665
:10F9A00069F736E47312F8C0963409F041C02C812F
:10F9B0003D816901E12CF12CCC0CDD1CEE1CFF1CFF
:10F9C00080910001A0E0B1E0B701A60111963C9141
:10F9D00011973A83198229813A81282BC90131E094
:10F9E0000C01FA0160935B0030935700E8951124F5
:10F9F0004E5F5F4F6F4F7F4F0250110929F01296F3
:10FA00008C9112971296E2CF85E0F601E0925B00AE
:10FA100080935700E89507B600FCFDCF6092570031
:10FA2000E89576956795579547955D834C83C2C059
:10FA3000953409F0BFC07801CC80DD8040E0A42E71
:10FA400041E0B42EF50161915F01C6010E9401FE03
:10FA5000FFEFCF1ADF0A21E0E21AF10899F72C81B3
:10FA60003D81200F311F3D832C83A4C0873609F0D0
:10FA700056C00E941BFC982E812C0E941BFC840106
:10FA8000082B0E941BFC863489F52C813D8159018D
:10FA9000C12CD12CAA0CBB1CCC1CDD1C3FEFA31627
:10FAA00037EFB30631E0C306D10428F4CBBEF5012D
:10FAB0008791969102C08FEF9FEF8B839E830E9468
:10FAC00014FC9E81892F0E9414FC82E0A80EB11CB8
:10FAD000C11CD11C0250110909F7D601C501B69508
:10FAE000A795979587959D838C831CCF853409F0C6
:10FAF00019CF7801CC80DD80C6010E94F9FD0E94FB
:10FB000014FC9FEFC91AD90AE1E0EE1AF108A1F737
:10FB10002C813D81200F311F3D832C8303CF8536FF
:10FB2000F1F436E4731246C080E090E0DC0123E09B
:10FB3000FC01A0935B0020935700E89507B600FCFA
:10FB4000FDCF9F5FAF4FBF4F811538EF930731E077
:10FB5000A307B10561F760925700E8952BC0853483
:10FB600061F488E190E0ECE00FB6F894A8958093FA
:10FB700060000FBEE09360001DC0803509F41AC01C
:10FB80008C3409F417C0803711F483E52FC0843713
:10FB900029F486E40E9414FC80E028C0982F98572E
:10FBA000923018F40E941BFC05C0843529F40E9491
:10FBB0001BFC782E8DE01AC0833519F40E9423FCBB
:10FBC000B1CE863529F480E30E9414FC88E30EC090
:10FBD000833741F485E00E9414FC87E90E9414FCFD
:10FBE0008EE104C08B3109F49DCE8FE30E9414FC9A
:10FBF00099CEF999FECF92BD81BDF89A992780B52B
:10FC00000895262FF999FECF1FBA92BD81BD20BD60
:10FC10000FB6F894FA9AF99A0FBE01960895F894DF
:02FC2000FFCF14
:040000031000F800F1
:00000001FF
